:020000040000FA
:0600000007EF2AF01200D8
:0620000007EF2AF01200B8
:062008004FEF27F012006B
:062018004FEF27F012005B
:02202A000000B4
:04202C00D9CFE6FF23
:10203000E1CFD9FFE652928092820D0EC16E030E5F
:10204000C06E9284809489949286809689969288B4
:102050008998899A929A8A9693968A889398938A6D
:10206000818AF19E8A9493948B9094908B9294920F
:102070008B949494949C8B8CDF6A400EDF5C10E20E
:10208000DF50EA6A010FE96E010EEA22EF6ADF50C3
:10209000EA6A410FE96E010EEA22EF6ADF2AEDD704
:1020A0000101816B0101020E826F0101030E836F3A
:1020B0000101040E846F0101050E856F0101060EFA
:1020C000866F0101080E876F0101180E886F0101EC
:1020D0000A0E896F0101090E8A6F01010B0E8B6FC9
:1020E00001018C6901018D6901018E6901018F690E
:1020F00001019069080ED56E040ECA6E4F0ECB6EAC
:102100000C0EBD6E1D0EBE6E0101400EE16F010191
:102110003E0EE26F01013C0EE36F01017E0E986FEF
:1021200001012D0E996F0101936B070EB46EB56A14
:10213000F28CF28E28EC27F0E552E552E7CFD9FF7A
:102140001200D9CFE6FFE1CFD9FF080EE126010149
:102150009A6B400EE66E010EE66E010EE66ED9EC4D
:1021600026F0E552E552E552000802E387EF1BF046
:10217000400E01019A5D02E387EF1BF001019A51C5
:10218000EA6A010FE96E010EEA22EF50420A02E10B
:1021900063EF1BF00F0A02E12EEF1BF03E0A02E193
:1021A000C8EF1AF0140A02E194EF1AF0130A02E1E0
:1021B00069EF1AF0E00A02E158EF1AF0070A02E1AB
:1021C00034EF1AF0010A02E12DEF1AF0030A02E1DE
:1021D00028EF1AF0010A02E120EF1AF0170A02E1D3
:1021E00048EF19F0030A02E174EF18F0060A02E161
:1021F000B3EF17F0070A02E11DEF17F0030A02E13F
:10220000BBEF16F0070A02E1E5EF15F0010A02E163
:1022100042EF15F0D30A01E1C0D3670A01E1EAD227
:102220007A0A01E185D2200A01E116D20A0A01E107
:10223000FCD1200A01E1E2D1330A01E1AED1200A4A
:1022400001E17AD1320A01E171D1200A01E168D1BC
:102250000C0A01E136D10A0A01E12DD1110A01E18E
:1022600024D1200A01E11BD1020A01E112D13F0A67
:1022700001E109D11F0A01E100D1260A01E1E3D001
:10228000200A01E193D0350A6EE0220A02E083EFD2
:102290001BF001019A2B01019A51EA6A010FE96EC4
:1022A000010EEA22EF50800B5AE0C050DE6EDD6A6C
:1022B0000A0EC16E01019A51EA6A010FE96E010E20
:1022C000EA22EF507F0B01019D6F01019A2B010162
:1022D0009A51EA6A010FE96E010EEA22EF50030BF0
:1022E000040DF328C26E860EC06E01019B6B0101C6
:1022F0009C6B01019D5101019B5D20E20A0EE66E7F
:1023000013EC2AF0E552C282C2B2FED79E9C0101B4
:102310009C519C2BEA6A410FE96E010EEA22C3CF61
:10232000EFFF01019C519C2BEA6A410FE96E010EFF
:10233000EA22C4CFEFFF01019B2BDBD704010CBFC6
:102340000BD0400EE66E410EE66E010EE66E9DEC81
:1023500026F0E552E552E5520D0EC16EC09E010118
:102360009A2B85EF1BF002C181F103C182F104C1F8
:1023700083F105C184F106C185F107C186F108C169
:1023800087F109C188F10AC189F10BC18AF10CC139
:102390008BF10DC18CF10EC18DF10FC18EF110C109
:1023A0008FF10101400E9A6F85EF1BF001019A2B0E
:1023B00001019A51EA6A010FE96E010EEA22EF501B
:1023C000040B1FE093EC1BF0050EC26E780EE66E58
:1023D000BCEC29F0E552C282C2B2FED79E9CC3CFAC
:1023E00041F1C4CF42F104010CBF0BD0400EE66EA8
:1023F000410EE66E010EE66E9DEC26F0E552E552CA
:10240000E55201019A51EA6A010FE96E010EEA22D2
:10241000EF50010B03E096EC1BF002D093EC1BF0A5
:1024200001019A51EA6A010FE96E010EEA22EF50AA
:10243000020B03E0A8EC22F002D0ACEC22F0010188
:102440009A2B85EF1BF00101010E416F0101140E63
:10245000426F0101436B04010CBF0BD0400EE66ECE
:10246000410EE66E010EE66E9DEC26F0E552E55259
:10247000E55201019A2B85EF1BF099EC1BF001014D
:102480009A2B85EF1BF0B5EC1BF001019A2B85EF21
:102490001BF0D1EC1BF001019A2B85EF1BF085ECB2
:1024A0001DF001019A2B85EF1BF0BEEC1DF0010120
:1024B0009A2B85EF1BF01EEC1EF001019A2B85EF85
:1024C0001BF001019A29EA6A010FE96E010EEA2266
:1024D000EF50DE6EDD6A020E01019A25EA6A010FF5
:1024E000E96E010EEA22EFCF0BF00C6A0BBE0C680E
:1024F0000BC00CF00B6AD9CFE9FFDACFEAFF0B5023
:10250000EE260C50ED22DECFE6FFDDCFE6FF59ECE4
:102510001DF0E552E552030E01019A2785EF1BF0ED
:1025200029EC1EF001019A2B85EF1BF033EC1EF015
:1025300001019A2B85EF1BF001019A29EA6A010F2C
:10254000E96E010EEA22EF50DE6EDD6A020E010135
:102550009A25EA6A010FE96E010EEA22EFCF0DF02B
:102560000E6A0DBE0E680DC00EF00D6ADE500D2411
:102570000B6EDD500E200C6E0BC0DEFF0CC0DDFFBD
:10258000DECFE6FFDDCFE6FF9AEC1EF0E552E55226
:10259000030E01019A2785EF1BF001019A29EA6ACF
:1025A000010FE96E010EEA22EF50DE6EDD6A020EC7
:1025B00001019A25EA6A010FE96E010EEA22EFCFC6
:1025C0000DF00E6A0DBE0E680DC00EF00D6ADE50E5
:1025D0000D240B6EDD500E200C6E0BC0DEFF0CC008
:1025E000DDFFDECFE6FFDDCFE6FFB4EC1EF0E55207
:1025F000E552030E01019A2785EF1BF001019A298C
:10260000EA6A010FE96E010EEA22EF50DE6EDD6A22
:10261000DECFE6FFDDCFE6FF5BEC1EF0E552E552D4
:10262000020E01019A2785EF1BF001019A29EA6A3F
:10263000010FE96E010EEA22EF50DE6EDD6ADECF99
:10264000E6FFDDCFE6FF7AEC1EF0E552E552020E22
:1026500001019A2785EF1BF001019A2B01019A5184
:102660009A2BEA6A010FE96E010EEA22EFCF9DF183
:1026700001019B6B01019D5101019B5D3CE2010148
:102680009B5105E086C1E6FFE5EC1BF0E552010138
:102690009A29EA6A010FE96E010EEA22EF503F0B18
:1026A0000B6E0C6A0BBE0C680BC0DEFF0CC0DDFFAE
:1026B000D9CFE9FFDACFEAFFEE50ED6EEF6A010104
:1026C0009A51EA6A010FE96E010EEA22EF50DF1219
:1026D00082C1E6FFE5EC1BF0E552DECFE6FFDDCF81
:1026E000E6FF1CEC1CF0E552E552020E01019A27B0
:1026F00001019B2BBFD788C1E6FFE5EC1BF0E5523B
:10270000030EE66EBCEC29F0E55289C1E6FFE5EC6C
:102710001BF0E5520C0EE66EF9EC29F0E55286C18D
:10272000E6FFE5EC1BF0E55228EC28F085EF1BF006
:1027300001019A2B01019A519A2BEA6A010FE96E65
:10274000010EEA22EFCF9DF101019B6B01019D512A
:1027500001019B5D3CE201019B5105E086C1E6FF62
:10276000E5EC1BF0E55201019A29EA6A010FE96ED6
:10277000010EEA22EF503F0B0B6E0C6A0BBE0C6889
:102780000BC0DEFF0CC0DDFFD9CFE9FFDACFEAFFD7
:10279000EE50ED6EEF6A01019A51EA6A010FE96E9F
:1027A000010EEA22EF50DF1282C1E6FFE5EC1BF0DA
:1027B000E552DECFE6FFDDCFE6FF1CEC1CF0E55274
:1027C000E552020E01019A2701019B2BBFD787C159
:1027D000E6FFE5EC1BF0E5520A0EE66EBCEC29F0D4
:1027E000E55286C1E6FFE5EC1BF0E55228EC28F047
:1027F00085EF1BF0020E01019A25EA6A010FE96ECE
:10280000010EEA22EF503F0B0B6E0C6A0BBE0C68F8
:102810000BC0DEFF0CC0DDFFD9CFE9FFDACFEAFF46
:10282000EE50ED6EEF6A01019A29EA6A010FE96E36
:10283000010EEA22EF50DF12040E01019A25EA6A26
:10284000010FE96E010EEA22EF503F0B0B6E0C6A8E
:102850000BBE0C68020E0BC0DBFF030E0CC0DBFFCF
:10286000D950020FE96EDACFEAFFEE50ED6EEF6A53
:10287000030E01019A25EA6A010FE96E010EEA22B0
:10288000EF500B6E0C6AD950020FE96EDACFEAFFF7
:102890000B50EE120C50ED12060E01019A25EA6A59
:1028A000010FE96E010EEA22EF503F0B0B6E0C6A2E
:1028B0000BBE0C68040E0BC0DBFF050E0CC0DBFF6B
:1028C000D950040FE96EDACFEAFFEE50ED6EEF6AF1
:1028D000050E01019A25EA6A010FE96E010EEA224E
:1028E000EF500B6E0C6AD950040FE96EDACFEAFF95
:1028F0000B50EE120C50ED12080E01019A25EA6AF7
:10290000010FE96E010EEA22EF503F0B0B6E0C6ACD
:102910000BBE0C68060E0BC0DBFF070E0CC0DBFF06
:10292000D950060FE96EDACFEAFFEE50ED6EEF6A8E
:10293000070E01019A25EA6A010FE96E010EEA22EB
:10294000EF500B6E0C6AD950060FE96EDACFEAFF32
:102950000B50EE120C50ED12060EDBCFE6FF070E09
:10296000DBCFE6FF040EDBCFE6FF050EDBCFE6FF95
:10297000020EDBCFE6FF030EDBCFE6FFDECFE6FF86
:10298000DDCFE6FFCFEC1EF0F56E080EE15EF550F0
:10299000090E01019A2785EF1BF001019A29EA6AC5
:1029A000010FE96E010EEA22EF50DE6EDD6A020EC3
:1029B00001019A25EA6A010FE96E010EEA22EFCFC2
:1029C0000DF00E6A0DBE0E680DC00EF00D6ADE50E1
:1029D0000D240B6EDD500E200C6E0BC0DEFF0CC004
:1029E000DDFF020EDBCFE6FF030EDBCFE6FFDECF1F
:1029F000E6FFDDCFE6FF2FEC22F0E552E552E5528F
:102A0000E552040EF3CFDBFF050EF4CFDBFFFF0E24
:102A1000E76E040EDBCF0BF0050EDBCF0CF0E750BA
:102A20000B160C6A0BC041F1D950040FE96EDACFD6
:102A3000EAFF080E0F0B06E0EC52D890ED32EF32B1
:102A4000E806FAE1FF0EE76E040EDBCF0BF0050E91
:102A5000DBCF0CF0E7500B160C6A0BC042F10401FF
:102A60000CBF0BD0400EE66E410EE66E010EE66E18
:102A70009DEC26F0E552E552E552050E01019A273C
:102A800085EF1BF001019A2B01019A519A2BEA6AFA
:102A9000010FE96E010EEA22EFCF9DF101019A517B
:102AA0009A2BEA6A010FE96E010EEA22EF50E66EF8
:102AB0000E0EE66EE66A1CEC1FF0E552E552E5529A
:102AC000F60EE66E6E0EE66EE66A1CEC1FF0E55240
:102AD000E552E55201019A519A2BEA6A010FE96E1B
:102AE000010EEA22EF50E66E0E0EE66EE66A1CEC70
:102AF0001FF0E552E552E552F70EE66E6E0EE66EF9
:102B0000E66A1CEC1FF0E552E552E55201019A51CC
:102B10009A2BEA6A010FE96E010EEA22EF50E66E87
:102B20000E0EE66EE66A1CEC1FF0E552E552E55229
:102B3000F80EE66E6E0EE66EE66A1CEC1FF0E552CD
:102B4000E552E552080EE66E82EC1FF0E5527CEC91
:102B50001CF0F3CFDEFFF4CFDDFF01019B6B010121
:102B60009D5101019B5D1FE2090EE66E82EC1FF094
:102B7000E5527CEC1CF0F3CFDEFFF4CFDDFFDECFBF
:102B80000BF0DDCF0CF0FF0E0B16000E0C16010142
:102B90009B51EA6A410FE96E010EEA220BC0EFFF7A
:102BA00001019B2BDCD704010CBFFDD7400EE66E64
:102BB000410EE66E010EE66E9DEC26F0E552E55202
:102BC000E55228EC28F085EF1BF001019A2B01015A
:102BD0009A519A2BEA6A010FE96E010EEA22EFCFB1
:102BE0009DF101019A519A2BEA6A010FE96E010EDB
:102BF000EA22EFCF0BF00C6A0BBE0C680BC0DEFFB5
:102C00000CC0DDFF01019A519A2BEA6A010FE96EAF
:102C1000010EEA22EFCF0BF00C6A0BBE0C68020E1D
:102C20000BC0DBFF030E0CC0DBFFA60EE66E9E0E94
:102C3000E66EE66A1CEC1FF0E552E552E552A60E80
:102C4000E66E9C0EE66EE66A1CEC1FF0E552E5525D
:102C5000E552020EDBCFE6FF0E0EE66EE66A1CECD6
:102C60001FF0E552E552E552AA0EE66E6E0EE66ED4
:102C7000E66A1CEC1FF0E552E552E55201019B6B40
:102C800001019D5101019B5D64E2DFCFE6FF0E0E65
:102C9000E66EE66A1CEC1FF0E552E552E552A90E1D
:102CA000E66E6E0EE66EE66A1CEC1FF0E552E5522B
:102CB000E552A60EE66E800EE66EE66A1CEC1FF08C
:102CC000E552E552E552A80EE66E500EE66EE66A53
:102CD0001CEC1FF0E552E552E552F50EE66E6E0E65
:102CE000E66EE66A1CEC1FF0E552E552E552A90ECD
:102CF000E66E6E0EE66EE66A1CEC1FF0E552E552DB
:102D0000E552020EE66E82EC1FF0E5527CEC1CF000
:102D1000060EF3CFDBFF070EF4CFDBFFFF0EE76EEF
:102D2000060EDBCF0BF0070EDBCF0CF0E7500B16D7
:102D30000C6A01019B51EA6A410FE96E010EEA2219
:102D40000BC0EFFFDF2A010E01E3DB2A01019B2B01
:102D500097D704010CBFFDD7400EE66E410EE66E1C
:102D6000010EE66E9DEC26F0E552E552E55228ECA8
:102D700028F085EF1BF001019A2B040EE66E0E0E73
:102D8000E66EE66A1CEC1FF0E552E552E552F60EDF
:102D9000E66E6E0EE66EE66A1CEC1FF0E552E5523A
:102DA000E552E66A0E0EE66EE66A1CEC1FF0E5528E
:102DB000E552E552F70EE66E6E0EE66EE66A1CEC24
:102DC0001FF0E552E552E5523C0EE66E0E0EE66E41
:102DD000E66A1CEC1FF0E552E552E552F80EE66E8D
:102DE0006E0EE66EE66A1CEC1FF0E552E552E55207
:102DF00001019A519A2BEA6A010FE96E010EEA224B
:102E0000EFCF9DF19DC1E6FFE66A0C0EE66E1CEC6D
:102E10001FF0E552E552E552E66AE66AE66A1CEC06
:102E20001FF0E552E552E552DEEC1FF0FA0EE66EB9
:102E3000BCEC29F0E55285EF1BF001019A2B050E41
:102E4000E66E0E0EE66EE66A1CEC1FF0E552E552E9
:102E5000E552F60EE66E6E0EE66EE66A1CEC1FF0AC
:102E6000E552E552E552E66A0E0EE66EE66A1CECA5
:102E70001FF0E552E552E552F70EE66E6E0EE66E75
:102E8000E66A1CEC1FF0E552E552E5523C0EE66E98
:102E90000E0EE66EE66A1CEC1FF0E552E552E552B6
:102EA000F80EE66E6E0EE66EE66A1CEC1FF0E5525A
:102EB000E552E55201019A29EA6A010FE96E010E15
:102EC000EA22EFCF9DF19DC1E6FF9DC1E6FF0C0E0A
:102ED000E66E1CEC1FF0E552E552E552E66AE66A42
:102EE000E66A1CEC1FF0E552E552E552040EE66E70
:102EF0000E0EE66EE66A1CEC1FF0E552E552E55256
:102F0000F60EE66E6E0EE66EE66A1CEC1FF0E552FB
:102F1000E552E55201019A51EA6A010FE96E010E8C
:102F2000EA22EFCF9DF19DC1E6FF9DC1E6FF0C0EA9
:102F3000E66E1CEC1FF0E552E552E552E66AE66AE1
:102F4000E66A1CEC1FF0E552E552E552DEEC1FF09C
:102F5000C80EE66EBCEC29F0E552020E01019A277C
:102F600028EC28F0D2D3A60EE66E8E0EE66EE66A48
:102F70001CEC1FF0E552E552E552A60EE66E9C0EE3
:102F8000E66EE66A1CEC1FF0E552E552E552020ED1
:102F900001019A25EA6A010FE96E010EEA22EF505B
:102FA000E66E0E0EE66EE66A1CEC1FF0E552E55288
:102FB000E552F60EE66E6E0EE66EE66A1CEC1FF04B
:102FC000E552E552E552030E01019A25EA6A010F26
:102FD000E96E010EEA22EF50E66E0E0EE66EE66A2C
:102FE0001CEC1FF0E552E552E552F70EE66E6E0E50
:102FF000E66EE66A1CEC1FF0E552E552E552040E5F
:1030000001019A25EA6A010FE96E010EEA22EF50EA
:10301000E66E0E0EE66EE66A1CEC1FF0E552E55217
:10302000E552F80EE66E6E0EE66EE66A1CEC1FF0D8
:10303000E552E552E55201019A29EA6A010FE96E6B
:10304000010EEA22EFCF9DF1050E01019A27010141
:103050009B6B01019D0501019B5D22E201019A51DB
:103060009A2BEA6A010FE96E010EEA22EFCF9FF177
:1030700001019A519A2BEA6A010FE96E010EEA22C8
:10308000EFCF9EF19FC1E6FF9EC1E6FF0D0EE66EFB
:103090001CEC1FF0E552E552E55201019B2BD9D7FC
:1030A00001019A519A2BEA6A010FE96E010EEA2298
:1030B000EFCF9FF101019A519A2BEA6A010FE96E55
:1030C000010EEA22EFCF9EF19FC1E6FF9EC1E6FF0F
:1030D0000F0EE66E1CEC1FF0E552E552E552ACEC2B
:1030E0001FF028EC28F011D3A60EE66E8E0EE66EC9
:1030F000E66A1CEC1FF0E552E552E552A60EE66EBC
:103100008C0EE66EE66A1CEC1FF0E552E552E552C5
:10311000A60EE66E840EE66EE66A1CEC1FF0E55223
:10312000E552E552E66AEF0EE66EE66A1CEC1FF029
:10313000E552E552E552E66AF80EE66EE66A1CECE8
:103140001FF0E552E552E552300EE66E0E0EE66EC9
:10315000E66A1CEC1FF0E552E552E552F80EE66E09
:103160006E0EE66EE66A1CEC1FF0E552E552E55283
:10317000E66A0E0EE66EE66A1CEC1FF0E552E552BA
:10318000E552F70EE66E6E0EE66EE66A1CEC1FF078
:10319000E552E552E55201019A2B01019A519A2B11
:1031A000EA6A010FE96E010EEA22EFCF9BF19BC1A3
:1031B000E6FF0E0EE66EE66A1CEC1FF0E552E552E5
:1031C000E552F60EE66E6E0EE66EE66A1CEC1FF039
:1031D000E552E552E55201019A519A2BEA6A010F34
:1031E000E96E010EEA22EFCF9FF101019A519A2B6D
:1031F000EA6A010FE96E010EEA22EFCF9EF19FC14C
:10320000E6FF9EC1E6FF0F0EE66E1CEC1FF0E552D6
:10321000E552E552ACEC1FF001019B2B9BC1E6FF90
:103220000E0EE66EE66A1CEC1FF0E552E552E55222
:10323000F60EE66E6E0EE66EE66A1CEC1FF0E552C8
:10324000E552E5529FC1E6FF9EC1E6FF0F0EE66E16
:103250001CEC1FF0E552E552E552ACEC1FF0E66ABB
:10326000E66AE66A1CEC1FF0E552E552E552E66AB2
:10327000E66AE66A1CEC1FF0E552E552E552E66AA2
:10328000E66AE66A1CEC1FF0E552E552E5523DD2D3
:10329000A60EE66E9E0EE66EE66A1CEC1FF0E55288
:1032A000E552E552A60EE66E9C0EE66EE66A1CEC52
:1032B0001FF0E552E552E552A60EE66E840EE66E6C
:1032C000E66A1CEC1FF0E552E552E55201019A292D
:1032D000EA6A010FE96E010EEA22EFCF9DF1020EBC
:1032E00001019A25EA6A010FE96E010EEA22EFCF89
:1032F0009FF1030E01019A25EA6A010FE96E010EA2
:10330000EA22EFCF9EF1040E01019A2701019B6B87
:1033100001019D5101019B5D01E385D09FC1E6FF45
:103320000E0EE66EE66A1CEC1FF0E552E552E55221
:10333000A90EE66E6E0EE66EE66A1CEC1FF0E55214
:10334000E552E5529EC1E6FF0E0EE66EE66A1CEC03
:103350001FF0E552E552E552AA0EE66E6E0EE66EDD
:10336000E66A1CEC1FF0E552E552E55201019A5164
:103370009A2BEA6A010FE96E010EEA22EF50E66E1F
:103380000E0EE66EE66A1CEC1FF0E552E552E552C1
:10339000A80EE66E6E0EE66EE66A1CEC1FF0E552B5
:1033A000E552E552550EE66E0E0EE66EE66A1CEC30
:1033B0001FF0E552E552E552A70EE66E6E0EE66E80
:1033C000E66A1CEC1FF0E552E552E552AA0EE66EE5
:1033D0000E0EE66EE66A1CEC1FF0E552E552E55271
:1033E000A70EE66E6E0EE66EE66A1CEC1FF0E55266
:1033F000E552E552A60EE66E820EE66EE66A1CEC1B
:103400001FF0E552E552E552E66AE66AE66A1CEC10
:103410001FF0E552E552E552DEEC1FF001019F2B53
:1034200001019B2B75D7A60EE66E940EE66EE66A3A
:103430001CEC1FF0E552E552E55228EC28F065D16E
:1034400026EC27F08B920BEC20F001019A2B5DD13A
:1034500066EC20F001019A2B58D176EC20F00101A6
:103460009A2B28EC28F051D101019A2B01019B6B7A
:10347000200E01019B5D18E201019A5101019B257B
:10348000EA6A010FE96E010EEA22EF50E66E0101D1
:103490009B51EA6AA00FE96E010EEA22E552E7505D
:1034A000EF6E01019B2BE4D7200E01019A272DD14D
:1034B00001019A2B9AC1E6FFA00EE66E010EE66EA0
:1034C0000CEC21F0E552E552E552230E01019A275A
:1034D0001CD1929689969294899401019A2B0101AC
:1034E0009A51EA6A010FE96E010EEA22EFCF9DF1CF
:1034F00001019B6B01019D5101019B5D10E20101E6
:103500009A2B01019A51EA6A010FE96E010EEA2233
:10351000EF50E66EC3D9E55201019B2BEBD79286A3
:10352000928401019A2BF1D0F29E01019A2B0101A4
:103530009A51EA6A010FE96E010EEA22EFCF9DF17E
:1035400001019B6B01019D5101019B5D0FE247DA77
:10355000E66E01019B51EA6A410FE96E010EEA2213
:10356000E552E750EF6E01019B2BECD7F28E040180
:103570000CBF0BD0400EE66E410EE66E010EE66EFD
:103580009DEC26F0E552E552E55201019A2BBDD0A3
:10359000020E01019A25EA6A010FE96E010EEA2284
:1035A000EF50BE6E01019A29EA6A010FE96E010E21
:1035B000EA22EF50E840E8403F0B0B6E0C6A0BBE6E
:1035C0000C680BC0DEFF0CC0DDFF300EDE16DD6ABE
:1035D000CF0EBD14BD6EBD500D6E0E6ADE500D10C7
:1035E0000B6EDD500E100C6E0B50BD6E030E010104
:1035F0009A25EA6A010FE96E010EEA22EFCFE1F1A6
:10360000040E01019A25EA6A010FE96E010EEA2211
:10361000EF280101E26F040E01019A25EA6A010F09
:10362000E96E010EEA22EF040101E36F050E0101CC
:103630009A25EA6A010FE96E010EEA22EFCF98F1AE
:10364000060E01019A25EA6A010FE96E010EEA22CF
:10365000EFCF99F1070E01019A2757D081A602D02A
:103660000101938181B802D00101938381A402D02A
:10367000010193859D50400B05E0C250020B02E012
:103680000101938B93C141F19D9C94C142F195C17D
:1036900043F196C144F197C145F19D8C0101936BB3
:1036A0003EEC27F004010CBF0BD0400EE66E410E3D
:1036B000E66E010EE66E9DEC26F0E552E552E5520F
:1036C00001019A2B22D026EC28F0840EA66EFE0E65
:1036D000F66E7F0EF76EF86AF56A0C00550EA76E4F
:1036E000AA0EA76EA6820101916B926B0101910750
:1036F000000E925B01019151921103E00000000065
:10370000F5D7FF0002D001019A2BB8EF10F0F56E4B
:10371000080EE15C02E2E16AE552E16EF550E55225
:10372000E7CFD9FF12008A888A8612008A968A9883
:1037300012008B80898A8A9422EC27F092968996CF
:1037400092948994780EE66EBCEC29F0E552899A41
:103750008A84120EE66E13EC2AF0E552E7DF010EC2
:10376000E66EBCEC29F0E55212008B80898A8A94BF
:1037700022EC27F09296899692948994780EE66EC0
:10378000BCEC29F0E552D2DF120EE66E13EC2AF003
:10379000E552899A8A84010EE66EBCEC29F0E55266
:1037A0001200C1DF780EE66E13EC2AF0E5528A941F
:1037B000898A0C0EE66EBCEC29F0E552899A26EC5B
:1037C00027F0928692848B901200D9CFE6FFE1CF4A
:1037D000D9FFE65292948996DF6A050EDF5C14E207
:1037E000FE0EDB50010BE8B08984E8A0899400004C
:1037F0008986FE0EDBCFF3FFF390F342FE0EF3CF8C
:10380000DBFF8996DF2AE9D7FE0EDB50010BE8B01B
:103810008984E8A0899400008986FE0EDBCFF3FF3F
:10382000F390F342FE0EF3CFDBFF92848996E552CC
:10383000E552E7CFD9FF1200D9CFE6FFE1CFD9FF9C
:10384000E6529294FD0EDBCFC0F1FE0EDBCFC1F14C
:103850008986DF6A0E0EDF5C10E289960101C05195
:10386000010B02E0898401D0899400008986D890F8
:103870000101C133C033DF2AEDD789960000000073
:103880008986000000008996020EE66E13EC2AF08D
:10389000E552E552E552E7CFD9FF1200D9CFE6FF56
:1038A000E1CFD9FFE652FE0EDBCFC2F1DF6A080E90
:1038B000DF5C17E289960C0EE66EF9EC29F0E55212
:1038C0000101C2A102D0898401D0899489860C0E9D
:1038D000E66EF9EC29F0E5520101C291C243DF2AFC
:1038E000E6D789960C0EE66EF9EC29F0E552E55222
:1038F000E552E7CFD9FF1200D9CFE6FFE1CFD9FFDC
:10390000E652DF6A080EDF5C0AE2898600000000EA
:1039100000008996000000000000DF2AF3D792849F
:103920000101C36BC46BDF6A080EDF5C14E2898699
:10393000000000000000D8900101C433C33380A40C
:1039400002D00101C38F0000899600000000000032
:103950000000DF2AE9D79294020EE66E13EC2AF0FB
:10396000E552C3C1F3FFC4C1F4FF00D0E552E552F4
:10397000E7CFD9FF1200D9CFE6FFE1CFD9FFE6525A
:1039800092840101C56BC66B898600000000899690
:10399000DF6A0E0EDF5C10E2898600000000000086
:1039A00080A402D00101C68D00008996D890010143
:1039B000C633C533DF2AEDD789860000000089961B
:1039C000020EE66E13EC2AF0E552C5C1F3FFC6C144
:1039D000F4FF00D0E552E552E7CFD9FF1200D9CF6E
:1039E000E6FFE1CFD9FF020EE1260101C76BC86BEC
:1039F000DF6A080EDF5C4EE2010EDB6A010EDB506F
:103A00000B6E0C6AD8900C5004E6FA0E0B5C000E9C
:103A10000C5809E280A604D0DE52FB0EDD6E02D007
:103A2000010EDB2AEBD7010EDB500B6E0C6AFA0E8F
:103A30000B1801E10C5002E1550E2FD0010EDB6A8C
:103A4000010EDB500B6E0C6AD8900C5004E6FA0E97
:103A50000B5C000E0C5809E280B604D0DE52FB0E5F
:103A6000DD6E02D0010EDB2AEBD7010EDB500B6EB0
:103A70000C6AFA0E0B1801E10C5002E1AA0E0DD0EF
:103A800080A402D00101C881D8900101C833C73396
:103A9000DF2AAFD70101C75100D0F56E020EE15CFD
:103AA00002E2E16AE552E16EF550E552E7CFD9FF57
:103AB0001200D9CFE6FFE1CFD9FF020EE126DE6A80
:103AC000DD6ADECF0BF0DDCF0CF0FD0EDBCF0DF0AD
:103AD000FE0EDBCF0EF00D500B5C0E500C5809E2C1
:103AE00086C1E6FF72DEE552DF2A010E01E3DB2A22
:103AF000E8D7F56E020EE15C02E2E16AE552E16EA2
:103B0000F550E552E7CFD9FF1200D9CFE6FFE1CF5C
:103B1000D9FFE652DF6A400EDF5C1BE285C1E6FF9B
:103B200054DEE55228DFF3CF0BF0F4CF0CF0FF0E9C
:103B30000B16000E0C16DF50EA6A410FE96E010EFB
:103B4000EA220BC0EFFF86C1E6FF3FDEE552DF2A27
:103B5000E2D704010CBFFDD7400EE66E410EE66EC3
:103B6000010EE66E9DEC26F0E552E552E55228EC9A
:103B700028F0E552E552E7CFD9FF1200D9CFE6FF92
:103B8000E1CFD9FF030EE126DF6A400EDF5C3AE2A7
:103B900084C1E6FF1ADEE552EEDEDE52F3CFDEFF31
:103BA000F4CFDDFFDD52FF0EE76E010EDBCF0BF031
:103BB000020EDBCF0CF0E7500B160C6ADF50DF2A49
:103BC000EA6A410FE96E010EEA220BC0EFFF010E17
:103BD000DBCF0BF0020EDBCF0CF00CC00BF00C6A4D
:103BE000FF0E0B16000E0C16DF50EA6A410FE96E4D
:103BF000010EEA220BC0EFFF86C1E6FFE6DDE552CB
:103C0000DF2AC3D704010CBFFDD7400EE66E410E7C
:103C1000E66E010EE66E9DEC26F0E552E552E552A9
:103C200028EC28F0F56E030EE15C02E2E16AE55251
:103C3000E16EF550E552E7CFD9FF120081C1E6FFF2
:103C4000C4DDE552000EE66EE66AF6DDE552E552A9
:103C500012008AC1E6FFB9DDE5520C0EE66EBCEC3F
:103C600029F0E55212008BC1E6FFAFDDE5520C0EE4
:103C7000E66EBCEC29F0E552120087C1E6FFA5DD37
:103C8000E552030EE66EBCEC29F0E552120088C145
:103C9000E6FF9BDDE552030EE66EBCEC29F0E55233
:103CA000120089C1E6FF91DDE5520C0EE66EF9ECDB
:103CB00029F0E5521200D9CFE6FFE1CFD9FF83C149
:103CC000E6FF83DDE552FD0EDBCFE6FFFE0EDBCF28
:103CD000E6FFB2DDE552E552D0DF050EE66EBCEC44
:103CE00029F0E55286C1E6FF70DDE552E552E7CFE7
:103CF000D9FF1200D9CFE6FFE1CFD9FF83C1E6FF9C
:103D000064DDE552FD0EDBCFE6FFFE0EDBCFE6FF06
:103D100093DDE552E552BBDF050EE66EBCEC29F003
:103D2000E552BFDF86C1E6FF50DDE552E552E7CF41
:103D3000D9FF1200D9CFE6FFE1CFD9FF82C1E6FF5C
:103D400044DDE552FD0EDBCFE6FFFE0EDBCFE6FFE6
:103D500073DDE552E55291DF86C1E6FF36DDE552BF
:103D6000E552E7CFD9FF1200D9CFE6FFE1CFD9FF67
:103D700082C1E6FF2ADDE552FD0EDBCFE6FFFE0E37
:103D8000DBCFE6FF59DDE552E55281DF8ADF86C1F0
:103D9000E6FF1BDDE552E552E7CFD9FF1200D9CF90
:103DA000E6FFE1CFD9FF82C1E6FF0FDDE552FD0E50
:103DB000DBCFE6FFFE0EDBCFE6FF3EDDE552E55250
:103DC00086C1E6FF02DDE55282C1E6FFFEDCE55278
:103DD000FB0EDBCFE6FFFC0EDBCFE6FF2DDDE55271
:103DE000E55286C1E6FFF1DCE55282C1E6FFEDDC7B
:103DF000E552F90EDBCFE6FFFA0EDBCFE6FF1CDD66
:103E0000E552E55286C1E6FFE0DCE55282C1E6FFFD
:103E1000DCDCE552F70EDBCFE6FFF80EDBCFE6FF8A
:103E20000BDDE552E55229DF86C1E6FFCEDCE55227
:103E3000E552E7CFD9FF1200D9CFE6FFE1CFD9FF96
:103E4000E652FE0EDB500101C96FCA6BDF6A040E39
:103E5000DF5C15E289960000000000000101C951F5
:103E6000010B02E0898401D089940000000089865A
:103E70000000D8900101CA33C933DF2AE8D7FC0E0D
:103E8000DB500101C96FCA6BDF6A080EDF5C15E207
:103E900089960000000000000101C951010B02E0F9
:103EA000898401D089940000000089860000D890A0
:103EB0000101CA33C933DF2AE8D7FD0EDB50010107
:103EC000C96FCA6BDF6A080EDF5C15E289960000D5
:103ED000000000000101C951010B02E0898401D0FA
:103EE00089940000000089860000D8900101CA333F
:103EF000C933DF2AE8D789968994E552E552E7CF9E
:103F0000D9FF1200D9CFE6FFE1CFD9FFE652FE0E6E
:103F1000DB500101CB6FCC6BDF6A040EDF5C15E276
:103F200089960000000000000101CB51010B02E066
:103F3000898401D089948986000000000000D8900F
:103F40000101CC33CB33DF2AE8D789968994E55237
:103F5000E552E7CFD9FF1200D9CFE6FFE1CFD9FF75
:103F6000E6528994DF6A040EDF5C0AE2899600005B
:103F7000000000008986000000000000DF2AF3D75F
:103F80000C0EE66EE9EC29F0E5528996780EE66EA5
:103F900013EC2AF0E552DF6A100EDF5C0AE2898634
:103FA0000000000000008996000000000000DF2AE9
:103FB000F3D7E552E552E7CFD9FF1200D9CFE6FF9C
:103FC000E1CFD9FFE6528994DF6A040EDF5C0AE292
:103FD00089960000000000008986000000000000B3
:103FE000DF2AF3D789963C0EE66EBCEC29F0E55249
:103FF000DF6A100EDF5C0AE2898600000000000024
:104000008996000000000000DF2AF3D7E552E55250
:10401000E7CFD9FF1200D9CFE6FFE1CFD9FF020EDB
:10402000E1268B808A94898A96EC1BF09296899679
:1040300092948994010EE66EBCEC29F0E552DE6A9A
:10404000DD6ADECF0BF0DDCF0CF0D8900C5004E62B
:10405000040E0B5C000E0C5813E28A84899A0C0E35
:10406000E66E13EC2AF0E5528A94898A010EE66E18
:10407000BCEC29F0E552DF2A010E01E3DB2AE1D78F
:10408000B20EE66E0BDCE552C20EE66E4EEC1CF094
:10409000E552120EE66E4EEC1CF0E5520A0EE66E8C
:1040A0004EEC1CF0E5528A84899A1E0EE66EBCEC3A
:1040B00029F0E552F56E020EE15C02E2E16AE5529A
:1040C000E16EF550E552E7CFD9FF120093EC1BF0FB
:1040D0008A94898A0C0EE66EBCEC29F0E552899A26
:1040E00026EC27F0928692848B901200050EE66EE5
:1040F0000E0EE66EE66AA0DEE552E552E552F60ED9
:10410000E66E6E0EE66EE66A97DEE552E552E55221
:10411000E66A0E0EE66EE66A8FDEE552E552E5527D
:10412000F70EE66E6E0EE66EE66A86DEE552E55244
:10413000E5523C0EE66E0E0EE66EE66A7DDEE55258
:10414000E552E552F80EE66E6E0EE66EE66A74DE35
:10415000E552E552E552010EE66E010EE66E0C0EDA
:10416000E66E6ADEE552E552E552040EE66E0E0E8C
:10417000E66EE66A61DEE552E552E552F60EE66E5F
:104180006E0EE66EE66A58DEE552E552E552800EA6
:10419000E66E800EE66E0C0EE66E4EDEE552E552E1
:1041A000E552E66AE66AE66A47DEE552E552E5521E
:1041B00001D81200D9CFE6FFE1CFD9FFE6528994AA
:1041C000DF6A040EDF5C0AE289960000000000004E
:1041D0008986000000000000DF2AF3D78996F00EE0
:1041E000E66EBCEC29F0E552F00EE66EBCEC29F070
:1041F000E552DF6A100EDF5C0AE2898600000000EB
:1042000000008996000000000000DF2AF3D7E55285
:10421000E552E7CFD9FF1200D9CFE6FFE1CFD9FFB2
:10422000030EE126A60EE66E840EE66EE66A04DE56
:10423000E552E552E552FC0EDBCFF3FFDB2AF350EB
:10424000EA6A010FE96E010EEA22EF50E66E0E0EE9
:10425000E66EE66AF1DDE552E552E552F60EE66EEF
:104260006E0EE66EE66AE8DDE552E552E552FC0EBA
:10427000DBCFF3FFDB2AF350EA6A010FE96E010E90
:10428000EA22EF50E66E0E0EE66EE66AD5DDE552E6
:10429000E552E552F70EE66E6E0EE66EE66ACCDD8E
:1042A000E552E552E552FC0EDBCFF3FFDB2AF3507B
:1042B000EA6A010FE96E010EEA22EF50E66E0E0E79
:1042C000E66EE66AB9DDE552E552E552F80EE66EB5
:1042D0006E0EE66EE66AB0DDE552E552E552DF6A43
:1042E000200EDF5C2DE2DF50E76EFD0EDBCFE9FF35
:1042F000FE0EDBCFEAFFE750E926000EEA22020EAF
:10430000EFCFDBFFDF28E76EFD0EDBCFE9FFFE0E10
:10431000DBCFEAFFE750E926000EEA22010EEFCFDD
:10432000DBFF020EDBCFE6FF010EDBCFE6FF0D0E5B
:10433000E66E82DDE552E552E552020EDF26D0D769
:10434000DF6A0F0EDF5C28E2FC0EDBCFF3FFDB2A17
:10435000F350EA6A010FE96E010EEA22020EEFCF76
:10436000DBFFFC0EDBCFF3FFDB2AF350EA6A010F21
:10437000E96E010EEA22010EEFCFDBFF020EDBCF6A
:10438000E6FF010EDBCFE6FF0D0EE66E55DDE552D2
:10439000E552E552DF2AD5D7FC0EDBCFF3FFDB2A4F
:1043A000F350EA6A010FE96E010EEA22020EEFCF26
:1043B000DBFFFC0EDBCFF3FFDB2AF350EA6A010FD1
:1043C000E96E010EEA22010EEFCFDBFF020EDBCF1A
:1043D000E6FF010EDBCFE6FF0F0EE66E2DDDE552A8
:1043E000E552E5520CD8F56E030EE15C02E2E16A9B
:1043F000E552E16EF550E552E7CFD9FF1200D9CF73
:10440000E6FFE1CFD9FFE6528994DF6A040EDF5C54
:104410000AE2899600000000000089860000000082
:104420000000DF2AF3D70C0EE66EBCEC29F0E55253
:104430008996000000000000DF6A100EDF5C0AE2CF
:10444000898600000000000089960000000000003E
:10445000DF2AF3D7E552E552E7CFD9FF1200D9CFD3
:10446000E6FFE1CFD9FF080EE126040EDB6A050E58
:10447000DB6A060EDB6A070EDB6AFD0EDBCF06F099
:10448000FE0EDBCF07F0020E06C0DBFF030E07C0F7
:10449000DBFFDE6ADD6ADECF0BF0DDCF0CF0020E53
:1044A000DBCF0DF0030EDBCF0EF00D500B5C0E508A
:1044B0000C5824E284C1E6FFE5EC1BF0E552BBECAE
:1044C0001CF0F3CF0BF0F4CF0CF00D6A0E6AD9504C
:1044D000040FE96EDACFEAFF0B50EE260C50EE2205
:1044E0000D50EE220E50EE2286C1E6FFE5EC1BF0E9
:1044F000E552DF2A010E01E3DB2ACDD7700EE66E0E
:10450000E5EC1BF0E552030EE66EBCEC29F0E5523B
:10451000D950040FE96EDACFEAFFEE52EE52EE6A9E
:10452000EE6A040EDBCF0BF0050EDBCF0CF00BC0F8
:10453000F3FF0CC0F4FF00D0F56E080EE15C02E260
:10454000E16AE552E16EF550E552E7CFD9FF12007E
:10455000D58E9298F28A1200D59EF29A9288899806
:1045600012008150200B01E0010E0101005D0AE004
:104570008150200B01E0010E0101006F81BA02D0D1
:10458000010E02D0000E00D01200D9CFE6FFE1CF1D
:10459000D9FF020EE126F56E020EE15C02E2E16A4D
:0E45A000E552E16EF550E552E7CFD9FF12006B
:0245AE006C504F
:1045B0000BE1040100513C0BE842E8420D0802E126
:1045C00008D801D03ED804D0040E6C5C01E14BD871
:1045D0001200D9CFE6FFE1CFD9FFE6520101D76B38
:1045E0000101D86B0101DD6BDE6B6FEC24F0DF6A3B
:1045F000DF500B6E0C6A010E0B5C000E0C581BE2B8
:104600000101D85101E017D0F76ADF34FE0BF7360D
:10461000F66ED80EF626520EF7220900F5CF0BF0F3
:104620000800F5CF0CF004D00CC0FAFF0B50F96E67
:10463000FBDFDF2ADDD7F4D8E552E552E7CFD9FF1B
:104640001200020E0101D75D0CE1A6D8040100BDE5
:1046500004D00401C80E006F03D00401880E006F5F
:1046600001D02DD91200040E0101E45D0CE112C449
:104670006EFF6E50000804E20101050EE46F03D0E6
:104680000101030EE46F0101D7050CE10DD804010F
:1046900004BD04D00401C80E046F03D00401880EC9
:1046A000046F01D00CD91200D9CFE6FFE1CFD9FFBA
:1046B000020EE1260101080EDD5D000EDE5905E265
:1046C000DDC1DEFFDEC1DDFF03D0080EDE6EDD6A78
:1046D0000401049304010491010EDB50040104134E
:1046E000DFCF05F4000EDB500101DD5F010EDB5072
:1046F0000101DE5B0101180EDB6F040EDC6F0101AE
:10470000E5A320D0D9CFE9FFDACFEAFFEE50ED10D4
:1047100018E0D9C1F6FFDAC1F7FF0800F550DBC198
:10472000E9FFDCC1EAFFEF6E0101DB2B000EDC23A9
:104730000101D92B000EDA23DF06010E01E2DB06B0
:10474000E1D71ED0D9CFE9FFDACFEAFFEE50ED1066
:1047500017E0D9C1E9FFDAC1EAFFEF50DBC1E9FF99
:10476000DCC1EAFFEF6E0101DB2B000EDC2301014F
:10477000D92B000EDA23DF06010E01E2DB06E2D7B9
:10478000F56E020EE15C02E2E16AE552E16EF5507F
:10479000E552E7CFD9FF1200D9CFE6FFE1CFD9FF2D
:1047A000020EE126030E04010015E76E010EE7CFAD
:1047B000DBFF01C4DFFFDE500101DD27DD50010119
:1047C000DE230101180ED96F040EDA6FD9CFE9FF8D
:1047D000DACFEAFFEE50ED1017E0D9C1E9FFDAC1F8
:1047E000EAFFEF50DBC1E9FFDCC1EAFFEF6E010138
:1047F000DB2B000EDC230101D92B000EDA23DF06B0
:10480000010E01E2DB06E2D7F56E020EE15C02E288
:10481000E16AE552E16EF550E552E7CFD9FF1200AB
:104820006D980101D8510FE10401080E016F0401D8
:10483000100E026F040E036F0401840E006F04015A
:10484000840E046F3BD0040110AF25D00101DD516F
:104850000401165D0101DE510401175904E216C47A
:10486000DDF117C4DEF120DF0101010ED76F040175
:10487000080E016F0401100E026F040E036F040195
:10488000800E006F0401180E066F040E076F0401FE
:10489000C80E046F13D00101020ED76F0401056B1F
:1048A0000401C80E046F0401080E016F0401180E04
:1048B000026F040E036F0401C80E006F12000101A5
:1048C000D76B0401080E016F0401100E026F040E75
:0E48D000036F0401880E006F0401046B1200D8
:0248DE000401D3
:1048E0001051600BE842E842E842E842E842000921
:1048F00001E058D004011151070A53E00B0A51E0BE
:10490000070A42E0010A2CE00B0A28E0020A26E02E
:10491000030A22E0080A12E0010A0EE00F0A0AE088
:10492000030A01E03ED00101010ED86F0101040E1F
:10493000E46F38D038D836D093D834D00101010E86
:10494000D86F0101E60ED96F010EDA6F0101E59310
:104950000101010EDD6F26D0ABD824D0FAD822D0C9
:104960000101010ED86F040114510101D96FDA6BF6
:10497000E70E0101D927010E0101DA230101E593B8
:104980000101010EDD6F0ED00101010ED86F04018F
:104990001451EA6AE70FE96E010EEA2212C4EFFF32
:1049A00001D000D01200800E0401105D58E1040116
:1049B0001351030A34E0010A10E0030A01E04DD06C
:1049C0000101010ED86F01018A0ED96F510EDA6F05
:1049D000120E0101DD6FDE6B40D00101010ED86FB8
:1049E00004011251F66EF76AD890F636F736CA0E01
:1049F000F626520EF7220900F5CFD9F10A00F5CFBD
:104A0000DAF1020E0101F76AD925F66EDA51F722C2
:104A10000900F5CFDDF10A00F5CFDEF11ED001016E
:104A2000010ED86F04011251F66EF76AD890F6366F
:104A3000F736CE0EF626520EF7220900F5CFD9F141
:104A40000A00F5CFDAF1D9C1F6FFDAC1F7FF0800A5
:104A5000F5500101DD6FDE6B00D00101E58312002E
:104A60000101010ED86F0F0EE66E710EE66E0F0E8D
:104A7000E66EB0EC28F0E552E552E552010EE66E26
:104A8000E70EE66E010EE66EB0EC28F0E552E55258
:104A9000E55212C4E6F10401125104E10101050ED0
:104AA000E46F05D00101060EE46F85EC26F01200DC
:104AB0000401186B0401196B040110511F0B020A49
:104AC00015E0030A0FE0010A01E035D00101010EF3
:104AD000D86F02D0040118810101E5A102D00401C0
:104AE000188329D00101010ED86F25D00101010ED4
:104AF000D86F040114510F0B080DF3500C6A000F0E
:104B00000B6E040E0C2204011451800B01E0010E07
:104B1000040DF35001010B24DB6F000E0C20DC6F41
:104B2000DBC1E9FFDCC1EAFFEF50040B03E0040145
:104B3000010E186F00D00101D8050AE10101180E1D
:104B4000D96F040EDA6F0101E5930101020EDD6FEA
:104B500012000401120511E1040110511F0B00099C
:104B60000CE10101010ED86F030E0401115D03E198
:104B70000101E58102D00101E591040112513EE1FC
:104B8000040110511F0B020839E1040114510F0BED
:104B9000000934E00101010ED86F040114510F0B1C
:104BA000080DF3500C6A000F0B6E040E0C2204016A
:104BB0001451800B01E0010E040DF35001010B2490
:104BC000DB6F000E0C20DC6F030E0401115D07E1AA
:104BD000840EDBC1E9FFDCC1EAFFEF6E0FD00401F8
:104BE00014AF06D0DBC1E9FFDCC1EAFFEF6A06D0F3
:0E4BF000880EDBC1E9FFDCC1EAFFEF6E1200A8
:024BFE000401B0
:104C000010511F0B010801E07DD00401145101E097
:104C100079D0060E0401115D2FE104011351230A1E
:104C200028E0010A13E0030A01E024D00101020E8A
:104C3000D86F0101E60505E10101AE0ED96F510EF5
:104C4000DA6F090E0101DD6FDE6B14D00101020E77
:104C5000D86F0101E60505E10101AD0ED96F520ED5
:104C6000DA6F0101E60504E11D0E0101DD6FDE6B67
:104C700001D000D00101E58304011051600BE8422E
:104C8000E842E842E842E842010801E03BD0040182
:104C900011510B0A31E0080A21E0090A19E0080A5B
:104CA00009E00B0A05E0080A01E02CD02CD82AD034
:104CB0002BD828D00101020ED86F0101E80ED96F60
:104CC000010EDA6F0101E5930101010EDD6F1AD0CB
:104CD0000101020ED86F13C4E8F114D00101020ED5
:104CE000D86F0101E90ED96F010EDA6F0101E5936A
:104CF0000101010EDD6F06D00101020ED86F12C452
:104D0000E9F100D01200120012000101EA6B1E0E40
:104D1000716E0401400E096F0401200E0A6F040E2B
:104D20000B6F0401880E086F0401600E0E6F040EF5
:104D30000F6F0401400E0C6F1200D9CFE6FFE1CFD8
:104D4000D9FFE652FC0EDB50400805E2400EF36E40
:104D5000FC0EF3CFDBFFDF6AFC0EDB50DF5C19E2F9
:104D6000DF50E76EFD0EDBCFE9FFFE0EDBCFEAFF83
:104D7000E750E926000EEA22EF50E66EDF50EA6ABD
:104D8000600FE96E040EEA22E552E750EF6EDF2A6B
:104D9000E3D7FC0EDBCF0DF4400E04010C17040129
:104DA0000C7D880E04010C13E552E552E7CFD9FFC4
:104DB0001200D9CFE6FFE1CFD9FF0101EA6B040170
:104DC00008BF39D0FC0EDBCF0BF004010951D880AD
:104DD0000B5403E2FC0E09C4DBFF0101EA6BFC0E7D
:104DE000DB500101EA5D1CE20101EA51EA6A200F91
:104DF000E96E040EEA22EF50E66E0101EA51E76E19
:104E0000FD0EDBCFE9FFFE0EDBCFEAFFE750E92620
:104E1000000EEA22E552E750EF6E0101EA2BDFD7E0
:104E20000401400E096F400E040108170401087DBB
:104E3000880E040108130101EA5100D0E552E7CFC2
:044E4000D9FF120084
:0C4E44008A940C0EBA6E1200BA6A1200BA
:104E5000050EC26E3E0EC06E0101DF6B0101E06BFC
:104E60009E9C9D8CC2821200C26A9D9C1200CF6AD9
:104E7000CE6AB10ECD6E9E909D8012009D909E9048
:104E8000CD6A8B9012008A888A94F1DF01019387A2
:104E900012008A948A88EBDF010193891200D8CF2F
:104EA000E4FFE0CFE4FFE46EDACFE4FFE2CFDAFF25
:104EB000E9CFE4FFEACFE4FFF6CFE4FFF7CFE4FF6A
:104EC000F5CFE4FFF3CFE4FFF4CFE4FFFACFE4FF44
:104ED00000EE00F00B0EE80403E3EECFE4FFFBD797
:104EE00000EE0BF0040EE80403E3EECFE4FFFBD783
:104EF000E652D9CFE6FFE1CFD9FFE6529EAC4BD0C8
:104F00009E9C050EC25C19E18150100B0DE1010160
:104F10009851C45C09E2080E0101DF5D02E1B3DFD4
:104F200002D00101DF2B02D00101DF6BC4CF95F16C
:104F3000C3CF94F1010EC26E2DD0C2042BE10C0E32
:104F4000BA6EBA500CE00101E251D880C45401E2BB
:104F5000BB6A0101E351C45C02E2E1C1BBFF8150C5
:104F6000040B10E08050200B0DE101019951C45C4D
:104F700009E2080E0101E05D02E18BDF02D00101D0
:104F8000E02B02D00101E06BC4CF97F1C3CF96F1C3
:104F9000050EC26EC282F2A406D0F2948978F60E93
:104FA000D76EBD0ED66E9E50010B05E09D50010BD5
:104FB00002E09E908B70E552E552E7CFD9FFE552B3
:104FC00000EE0EF0040EE80403E3E5CFEDFFFBD79F
:104FD00000EE0AF00B0EE80403E3E5CFEDFFFBD78C
:104FE000E5CFFAFFE5CFF4FFE5CFF3FFE5CFF5FF1F
:104FF000E5CFF7FFE5CFF6FFE5CFEAFFE5CFE9FF25
:10500000E5CFDAFFE550E5CFE0FFE5CFD8FF1000B0
:105010006DA610D802D06DB614D80101E40509E1DF
:105020006DBA07D0686A696A698069880101020EF1
:10503000E46F12006D6A696A6D860101010EE46F0A
:1050400012006D6A696A0101E46B1200FADF120056
:105050000101E45101E13AD06850040B04E06950C9
:10506000040B01E038D86DB231D06850010B04E078
:105070006950010B01E052D86850100B04E06950F0
:10508000100B01E024D86850400B04E06950400B3D
:1050900001E039D86850200B04E06950200B01E092
:1050A00034D86850020B04E06950020B01E034D898
:1050B000030E0101E45D01E209D06850080B06E02F
:1050C0006950080B03E0D7EC22F06896120069845F
:1050D00068986D8212006D926994689412000101C3
:1050E000E5A110D0F8DF6D840101080EEB6F070E0B
:1050F000EC6F0101EB07000EEC5B0101EB51EC11D1
:10510000F8E16D941200689C120070A003D05FEC6F
:1051100024F07090689A1200689212006A6A686AB5
:105120009F0E6B6E7B0E696E6E6A0F0EE66E710ED1
:10513000E66E0F0EE66E14D8E552E552E552160EF5
:10514000706E68A602D06896FCD76D985FEC24F06C
:105150000101E5910101E66B0101030EE46F12000C
:10516000D9CFE6FFE1CFD9FFFD0EDBCFE9FFFE0E81
:10517000DBCFEAFFFC0EDB5004E0EE6AFC0EDB0640
:0A518000F9D7E552E7CFD9FF12007E
:06518A001201000200000A
:105190000008D804330001000102030209022900BB
:1051A000010102803209040000020300000009210D
:1051B00001000001221D00070581034000010705D1
:1051C00001034000010902200001020480320904A9
:1051D000000002FF000000070581034000010705F1
:1051E00001034000010403090434034D0069006316
:1051F0000072006F006300680069007000200054B6
:10520000006500630068006E006F006C006F00674F
:10521000007900200049006E0063002E0048035012
:1052200000490043006B0069007400200032002038
:10523000004D006900630072006F0063006F006E34
:1052400000740072006F006C006C0065007200203A
:1052500000500072006F006700720061006D006D09
:105260000065007200160350004900430031003809
:10527000004600320035003500300032035000494E
:105280000043006B006900740020003200200043DE
:10529000006F006E006600690067007500720061B3
:1052A00000740069006F006E00200032000600FFED
:1052B0000901A10119012940150026FF0075089573
:1052C000408102190129409102C09C51C551E5510C
:0A52D000E9511D5265527B52FE4B5E
:0652DA002A0EF66E200E04
:1052E000F76E000EF86E01010900F550D26F09004B
:1052F000F550D36F03E1D26701D03DD00900F550DE
:10530000CD6F0900F550CE6F0900F550CF6F090041
:105310000900F550E96E0900F550EA6E0900090030
:105320000900F550D06F0900F550D16F0900090050
:10533000F6CFD4F1F7CFD5F1F8CFD6F1CDC1F6FF46
:10534000CEC1F7FFCFC1F8FF0101D05302E1D15325
:1053500007E00900F550EE6ED007F8E2D107F9D763
:10536000D4C1F6FFD5C1F7FFD6C1F8FF0101D207BE
:08537000000ED35BBFD7120051
:08537800FF0EE350106EEF0E72
:1053800001D0F30EE76EE72EC3EF29F00C0E0F6E7F
:10539000E76AE72EC9EF29F00F2EC8EF29F0102E8B
:0653A000C1EF29F012002C
:0A53A60005D80FD8A1EC10F0FCD7D9
:1053B0001200140E6F6E0101E46B0101E56B010137
:1053C000E66B16EC10F0120008EC28F028EC28F040
:0253D0001200C9
:0E53D200FF0EE350106E480E01D04C0EE76E39
:1053E000E72EFED7E76AE72EFED7102EF7D700008C
:0253F0001200A9
:0E53F200FF0EE350106E1B0E00D001D0200EF7
:0E540000E76EE72EFED7102EFAD700D012006E
:02540E0013EE9B
:1054100000F023EE00F0F86A0A9C6DEC29F0D3EC62
:0654200029F0FDD7120087
:0A542600FF0EE350E84E12000000F4
:0C54300000D000D000D0E82EFAD7120007
:00000001FF
